 sgx_blit_test

 Timestamp is 4be8c2c7 (Tue May 11 11:36:55 2010)

 Preferred load address is 00010000

 Start         Length     Name                   Class
 0001:00000000 00000004H .CRT$XCA                CODE
 0001:00000004 00000004H .CRT$XCZ                CODE
 0001:00000008 00000004H .CRT$XIA                CODE
 0001:0000000c 00000004H .CRT$XIZ                CODE
 0001:00000010 00000004H .CRT$XPA                CODE
 0001:00000014 00000004H .CRT$XPZ                CODE
 0001:00000018 00000004H .CRT$XTA                CODE
 0001:0000001c 00000004H .CRT$XTZ                CODE
 0001:00000020 00000d20H .rdata                  CODE
 0001:00000d40 0000002aH .rdata$debug            CODE
 0001:00000d6c 000018e8H .text                   CODE
 0001:00002654 00000018H .xdata                  CODE
 0001:0000266c 00000028H .idata$2                CODE
 0001:00002694 00000014H .idata$3                CODE
 0001:000026a8 000000acH .idata$4                CODE
 0001:00002754 0000013aH .idata$6                CODE
 0001:0000288e 00000000H .edata                  CODE
 0002:00000000 000000acH .idata$5                DATA
 0002:000000ac 00000008H .data                   DATA
 0002:000000b4 00000010H .bss                    DATA
 0003:00000000 00000080H .pdata                  DATA

  Address         Publics by Value              Rva+Base       Lib:Object

 0000:00000000       ___safe_se_handler_count   00000000     <absolute>
 0000:00000000       ___safe_se_handler_table   00000000     <absolute>
 0001:00000000       __xc_a                     00011000     corelib0:crt0init.obj
 0001:00000004       __xc_z                     00011004     corelib0:crt0init.obj
 0001:00000008       __xi_a                     00011008     corelib0:crt0init.obj
 0001:0000000c       __xi_z                     0001100c     corelib0:crt0init.obj
 0001:00000010       __xp_a                     00011010     corelib0:crt0init.obj
 0001:00000014       __xp_z                     00011014     corelib0:crt0init.obj
 0001:00000018       __xt_a                     00011018     corelib0:crt0init.obj
 0001:0000001c       __xt_z                     0001101c     corelib0:crt0init.obj
 0001:0000003c       ??_C@_0BD@FOHFKAOE@INVALID?5ERROR?5CODE?$AA@ 0001103c     sgx_blit_test.obj
 0001:00000050       ??_C@_09KMCHPOPM@PVRSRV_OK?$AA@ 00011050     sgx_blit_test.obj
 0001:0000005c       ??_C@_0BF@KHEAJDEG@PVRSRV_ERROR_GENERIC?$AA@ 0001105c     sgx_blit_test.obj
 0001:00000074       ??_C@_0BL@BOENCAIM@PVRSRV_ERROR_OUT_OF_MEMORY?$AA@ 00011074     sgx_blit_test.obj
 0001:00000090       ??_C@_0BN@IHBDMIPO@PVRSRV_ERROR_TOO_FEW_BUFFERS?$AA@ 00011090     sgx_blit_test.obj
 0001:000000b0       ??_C@_0BO@EGNEIFEA@PVRSRV_ERROR_SYMBOL_NOT_FOUND?$AA@ 000110b0     sgx_blit_test.obj
 0001:000000d0       ??_C@_0BL@BKMGFOLH@PVRSRV_ERROR_OUT_OF_HSPACE?$AA@ 000110d0     sgx_blit_test.obj
 0001:000000ec       ??_C@_0BM@LGNAOM@PVRSRV_ERROR_INVALID_PARAMS?$AA@ 000110ec     sgx_blit_test.obj
 0001:00000108       ??_C@_0BN@MGJEIKFE@PVRSRV_ERROR_TILE_MAP_FAILED?$AA@ 00011108     sgx_blit_test.obj
 0001:00000128       ??_C@_0BK@JHPIKHJG@PVRSRV_ERROR_INIT_FAILURE?$AA@ 00011128     sgx_blit_test.obj
 0001:00000144       ??_C@_0CE@POPMCOCG@PVRSRV_ERROR_CANT_REGISTER_CALLB@ 00011144     sgx_blit_test.obj
 0001:00000168       ??_C@_0BM@COIEDMNF@PVRSRV_ERROR_INVALID_DEVICE?$AA@ 00011168     sgx_blit_test.obj
 0001:00000184       ??_C@_0BH@OEOFFCIM@PVRSRV_ERROR_NOT_OWNER?$AA@ 00011184     sgx_blit_test.obj
 0001:0000019c       ??_C@_0BJ@PHFCJIBD@PVRSRV_ERROR_BAD_MAPPING?$AA@ 0001119c     sgx_blit_test.obj
 0001:000001b8       ??_C@_0BF@KGIMOMJE@PVRSRV_ERROR_TIMEOUT?$AA@ 000111b8     sgx_blit_test.obj
 0001:000001d0       ??_C@_0BI@CDPBDDFH@PVRSRV_ERROR_NO_PRIMARY?$AA@ 000111d0     sgx_blit_test.obj
 0001:000001e8       ??_C@_0BP@FMELGOJO@PVRSRV_ERROR_FLIP_CHAIN_EXISTS?$AA@ 000111e8     sgx_blit_test.obj
 0001:00000208       ??_C@_0BN@JMHJCLJP@ERROR_CANNOT_ACQUIRE_SYSDATA?$AA@ 00011208     sgx_blit_test.obj
 0001:00000228       ??_C@_0BL@JPEIBKNH@PVRSRV_ERROR_SCENE_INVALID?$AA@ 00011228     sgx_blit_test.obj
 0001:00000244       ??_C@_0BK@JAAFMMBM@PVRSRV_ERROR_STREAM_ERROR?$AA@ 00011244     sgx_blit_test.obj
 0001:00000260       ??_C@_0DP@FHJOPEMA@PVRSRV_ERROR_INVALID_INTERRUPTPV@ 00011260     sgx_blit_test.obj
 0001:000002a0       ??_C@_0BP@PFBLKCEO@PVRSRV_ERROR_CMD_NOT_PROCESSED?$AA@ 000112a0     sgx_blit_test.obj
 0001:000002c0       ??_C@_0BJ@PHLIKBPN@PVRSRV_ERROR_CMD_TOO_BIG?$AA@ 000112c0     sgx_blit_test.obj
 0001:000002dc       ??_C@_0CE@FHHHLEGE@PVRSRV_ERROR_DEVICE_REGISTER_FAI@ 000112dc     sgx_blit_test.obj
 0001:00000300       ??_C@_0BI@JBKNPCOM@PVRSRV_ERROR_FIFO_SPACE?$AA@ 00011300     sgx_blit_test.obj
 0001:00000318       ??_C@_0BJ@IIGHNIEG@PVRSRV_ERROR_TA_RECOVERY?$AA@ 00011318     sgx_blit_test.obj
 0001:00000334       ??_C@_0BN@BKNBJNB@PVRSRV_ERROR_INDOSORLOWPOWER?$AA@ 00011334     sgx_blit_test.obj
 0001:00000354       ??_C@_0BM@MCHBLHIP@PVRSRV_ERROR_TOOMANYBUFFERS?$AA@ 00011354     sgx_blit_test.obj
 0001:00000370       ??_C@_0BL@FINKNLDE@PVRSRV_ERROR_NOT_SUPPORTED?$AA@ 00011370     sgx_blit_test.obj
 0001:0000038c       ??_C@_0CA@KIDKOOGL@PVRSRV_ERROR_PROCESSING_BLOCKED?$AA@ 0001138c     sgx_blit_test.obj
 0001:000003ac       ??_C@_0CA@NBGAMPKE@PVRSRV_ERROR_CANNOT_FLUSH_QUEUE?$AA@ 000113ac     sgx_blit_test.obj
 0001:000003cc       ??_C@_0CE@NLLBGAEA@PVRSRV_ERROR_CANNOT_GET_QUEUE_SP@ 000113cc     sgx_blit_test.obj
 0001:000003f0       ??_C@_0CG@FCILKACH@PVRSRV_ERROR_CANNOT_GET_RENDERDE@ 000113f0     sgx_blit_test.obj
 0001:00000418       ??_C@_0BD@COEEPPOL@PVRSRV_ERROR_RETRY?$AA@ 00011418     sgx_blit_test.obj
 0001:0000042c       ??_C@_0BJ@IMBALOKG@PVRSRV_DEVICE_ID_UNKNOWN?$AA@ 0001142c     sgx_blit_test.obj
 0001:00000448       ??_C@_0BH@OGEGGGCD@PVRSRV_DEVICE_ID_MSVDX?$AA@ 00011448     sgx_blit_test.obj
 0001:00000460       ??_C@_0BF@BBCLGMON@PVRSRV_DEVICE_ID_SGX?$AA@ 00011460     sgx_blit_test.obj
 0001:00000478       ??_C@_0CD@BDGFMHBG@PVRSRV_DEVICE_TYPE_EXT?5?$CI3rd?5Part@ 00011478     sgx_blit_test.obj
 0001:0000049c       ??_C@_0BE@GEDKFGMC@Not?5recognised?50x?$CFx?$AA@ 0001149c     sgx_blit_test.obj
 0001:000004b0       ??_C@_0BI@ICLDLMDM@?4?4?4?4?5ui32ProcessID?3?$CFlu?6?$AA@ 000114b0     sgx_blit_test.obj
 0001:000004c8       ??_C@_0DH@IDEKHJEN@?9?9?9?9?9?9?9?9?9?9?9?9?9?9?9?9?9?9?9?9?9?9?9?9?5End?5?9?9?9@ 000114c8     sgx_blit_test.obj
 0001:00000500       ??_C@_0BD@NOILHFAN@PVRSRVDisconnect?3?6?$AA@ 00011500     sgx_blit_test.obj
 0001:00000514       ??_C@_0BH@LMCBNGLN@SGXReleaseClientInfo?3?6?$AA@ 00011514     sgx_blit_test.obj
 0001:0000052c       ??_C@_0CF@DBFHMBAF@Display?5Class?5API?3?5close?5the?5dev@ 0001152c     sgx_blit_test.obj
 0001:00000554       ??_C@_0CM@LDEJMMMA@Attempt?5to?5destroy?5memory?5contex@ 00011554     sgx_blit_test.obj
 0001:00000580       ??_C@_0DD@GODBIEMM@Display?5Class?5API?3?5unmap?5display@ 00011580     sgx_blit_test.obj
 0001:000005b4       ??_C@_0BP@GJLKNMBD@Destroy?5the?5transfer?5context?3?6?$AA@ 000115b4     sgx_blit_test.obj
 0001:000005d4       ??_C@_0BK@JEPLKMMD@Free?5the?5source?5surface?3?6?$AA@ 000115d4     sgx_blit_test.obj
 0001:000005f0       ??_C@_0DM@HDFMECLL@Do?5a?5SRCCOPY?5blit?5to?5the?5top?5lef@ 000115f0     sgx_blit_test.obj
 0001:00000630       ??_C@_0EF@LPOGHLKJ@?$CItop?5left?5quadrant?5should?5be?5str@ 00011630     sgx_blit_test.obj
 0001:00000678       ??_C@_0DJ@OPOMFNMC@Polling?5for?5destination?5surface?5@ 00011678     sgx_blit_test.obj
 0001:000006b8       ??_C@_0EA@GMKAPJCA@Do?5a?5SRCCOPY?5blit?5to?5the?5bottom?5@ 000116b8     sgx_blit_test.obj
 0001:000006f8       ??_C@_0DL@IBIGKNM@?$CIbottom?5right?5quadrant?5should?5be@ 000116f8     sgx_blit_test.obj
 0001:00000738       ??_C@_0EE@NCNDJNKK@Display?5Class?5API?3?5ERROR?5unsuppo@ 00011738     sgx_blit_test.obj
 0001:0000077c       ??_C@_0CN@CJJNALAI@Attempt?5to?5create?5transfer?5conte@ 0001177c     sgx_blit_test.obj
 0001:000007ac       ??_C@_0CP@IFAFGPME@Display?5Class?5API?3?5map?5display?5s@ 000117ac     sgx_blit_test.obj
 0001:000007e0       ??_C@_0EK@BPNJOJAB@?4?4?4?4?5Shared?5heap?5?$CFlu?5?9?5HeapID?30x@ 000117e0     sgx_blit_test.obj
 0001:0000082c       ??_C@_0DE@BODOPOHG@Display?5Class?5API?3?5get?5the?5syste@ 0001182c     sgx_blit_test.obj
 0001:00000860       ??_C@_0ED@NNKEOJPF@?4?4?4?4?5Display?5dimensions?5?$CFlu?5?9?5By@ 00011860     sgx_blit_test.obj
 0001:000008a4       ??_C@_0DB@DPDHNDGF@Display?5Class?5API?3?5enumerate?5dis@ 000118a4     sgx_blit_test.obj
 0001:000008d8       ??_C@_0CK@PAKBMFJN@?4?4?4?4?5Display?5format?5?$CFlu?5?9?5Pixelf@ 000118d8     sgx_blit_test.obj
 0001:00000904       ??_C@_0O@GDPIEJBG@?4?4?4?4?5Name?3?$CFs?6?$AA@ 00011904     sgx_blit_test.obj
 0001:00000914       ??_C@_0BI@BLGHILNJ@?4?4?4?4?5MaxSwapChains?3?$CFlu?6?$AA@ 00011914     sgx_blit_test.obj
 0001:0000092c       ??_C@_0BO@POAFDAJE@?4?4?4?4?5MaxSwapChainBuffers?3?$CFlu?6?$AA@ 0001192c     sgx_blit_test.obj
 0001:0000094c       ??_C@_0BK@CPCAOBID@?4?4?4?4?5MinSwapInterval?3?$CFlu?6?$AA@ 0001194c     sgx_blit_test.obj
 0001:00000968       ??_C@_0BK@DMGFAHCI@?4?4?4?4?5MaxSwapInterval?3?$CFlu?6?$AA@ 00011968     sgx_blit_test.obj
 0001:00000984       ??_C@_0CO@GIPBIACE@Display?5Class?5API?3?5enumerate?5dis@ 00011984     sgx_blit_test.obj
 0001:000009b4       ??_C@_0CF@FMDFFMKC@Display?5Class?5API?3?5Get?5display?5i@ 000119b4     sgx_blit_test.obj
 0001:000009dc       ??_C@_0CA@DAONOMAK@Display?5Class?5API?3?5open?5device?6?$AA@ 000119dc     sgx_blit_test.obj
 0001:000009fc       ??_C@_0CL@DNLHEBLI@Attempt?5to?5create?5memory?5context@ 000119fc     sgx_blit_test.obj
 0001:00000a28       ??_C@_0CA@DGGJNKGO@?5Test?5Memory?5Allocation?5FAILED?6?$AA@ 00011a28     sgx_blit_test.obj
 0001:00000a48       ??_C@_0DM@CIPNLPOO@PVRSRVEnumerateDeviceClass?$CI?$CJ?5ret@ 00011a48     sgx_blit_test.obj
 0001:00000a84       ??_C@_0CG@MMBLEMBO@Display?5Class?5API?3?5enumerate?5dev@ 00011a84     sgx_blit_test.obj
 0001:00000aac       ??_C@_0BJ@NLALCGOE@Getting?5SGX?5Client?5info?6?$AA@ 00011aac     sgx_blit_test.obj
 0001:00000ac8       ??_C@_0BP@IDIGABKI@Attempt?5to?5acquire?5device?5?$CFd?3?6?$AA@ 00011ac8     sgx_blit_test.obj
 0001:00000ae8       ??_C@_0BH@PPGIPGOP@?5?5?5?5?5?5?5?5?5?5?5?5?$CF04d?5?5?5?5?$HM?5?$AA@ 00011ae8     sgx_blit_test.obj
 0001:00000b00       ??_C@_01EEMJAFIK@?6?$AA@   00011b00     sgx_blit_test.obj
 0001:00000b04       ??_C@_0BK@GEDDINJE@?4?4?4?4?5Reported?5?$CFu?5devices?6?$AA@ 00011b04     sgx_blit_test.obj
 0001:00000b20       ??_C@_0CD@INKLJIDI@?4?4?4?4?5Device?5Number?5?5?$HM?5Device?5Typ@ 00011b20     sgx_blit_test.obj
 0001:00000b44       ??_C@_04LNELOFCG@?5OK?6?$AA@ 00011b44     sgx_blit_test.obj
 0001:00000b4c       ??_C@_0DE@KAFOOJDI@Get?5number?5of?5devices?5from?5PVRSR@ 00011b4c     sgx_blit_test.obj
 0001:00000b80       ??_C@_0M@FBGHFOFL@?5FAIL?5?9?5?$CFs?6?$AA@ 00011b80     sgx_blit_test.obj
 0001:00000b8c       ??_C@_0DH@NPPDEKDN@?9?9?9?9?9?9?9?9?9?9?9?9?9?9?9?9?9?9?5SGX?53D?5Blit?5t@ 00011b8c     sgx_blit_test.obj
 0001:00000bc4       ??_C@_0DH@PPPHAACG@?9?9?9?9?9?9?9?9?9?9?9?9?9?9?9?9?9?9?9?9?9?9?9?5Start?5?9?9@ 00011bc4     sgx_blit_test.obj
 0001:00000bfc       ??_C@_0CL@KFFMIBHA@Call?5PVRSRVConnect?5with?5a?5valid?5@ 00011bfc     sgx_blit_test.obj
 0001:00000c28       ??_C@_1KE@BDGMONOJ@?$AAH?$AA?3?$AA?2?$AAW?$AAI?$AAN?$AAC?$AAE?$AA6?$AA0?$AA0?$AA?2?$AAP?$AAL?$AAA?$AAT?$AAF?$AAO?$AAR?$AAM?$AA?2?$AAS?$AAM?$AAD?$AAK?$AAV?$AA2?$AA1?$AA0?$AA?2?$AAS?$AAR@ 00011c28     wince_unittests.obj
 0001:00000ccc       ??_C@_1CI@OHCJFJPM@?$AAE?$AAR?$AAR?$AAO?$AAR?$AA?3?$AA?5?$AA?$CF?$AAs?$AA?5?$AAl?$AAi?$AAn?$AAe?$AA?5?$AA?$CF?$AAd?$AA?3?$AA?5?$AA?$AA@ 00011ccc     wince_unittests.obj
 0001:00000cf4       ??_C@_1CK@MPGKAOE@?$AA?$CI?$AAe?$AAr?$AAr?$AAo?$AAr?$AA?5?$AAc?$AAo?$AAd?$AAe?$AA?3?$AA?5?$AA?$CF?$AAd?$AA?$CJ?$AA?3?$AA?5?$AA?$CF?$AAs?$AA?$AA@ 00011cf4     wince_unittests.obj
 0001:00000d20       ??_C@_1M@DMCDIEDK@?$AAP?$AAK?$AAM?$AA1?$AA?3?$AA?$AA@ 00011d20     wince_unittests.obj
 0001:00000d2c       ??_C@_0L@GPAGIAIC@?9disablepm?$AA@ 00011d2c     wince_unittests.obj
 0001:00000d38       ??_C@_07FBLHGNAH@app?4exe?$AA@ 00011d38     wince_unittests.obj
 0001:00000f28       print_dev_type             00011f28 f   sgx_blit_test.obj
 0001:00000f88       main                       00011f88 f   sgx_blit_test.obj
 0001:00001e4c       WinMain                    00012e4c f   wince_unittests.obj
 0001:00002074       ReleasePowerRequirement    00013074 f   coredll:COREDLL.dll
 0001:00002084       NKDbgPrintfW               00013084 f   coredll:COREDLL.dll
 0001:00002094       FormatMessageW             00013094 f   coredll:COREDLL.dll
 0001:000020a4       GetLastError               000130a4 f   coredll:COREDLL.dll
 0001:000020b4       SetPowerRequirement        000130b4 f   coredll:COREDLL.dll
 0001:000020c4       WideCharToMultiByte        000130c4 f   coredll:COREDLL.dll
 0001:000020d4       PVRSRVDisconnect           000130d4 f   srvclum:SRVCLUM.dll
 0001:000020e4       SGXReleaseClientInfo       000130e4 f   srvclum:SRVCLUM.dll
 0001:000020f4       PVRSRVCloseDCDevice        000130f4 f   srvclum:SRVCLUM.dll
 0001:00002104       PVRSRVDestroyDeviceMemContext 00013104 f   srvclum:SRVCLUM.dll
 0001:00002114       PVRSRVUnmapDeviceClassMemory 00013114 f   srvclum:SRVCLUM.dll
 0001:00002124       SGXDestroyTransferContext  00013124 f   srvclum:SRVCLUM.dll
 0001:00002134       PVRSRVFreeDeviceMem        00013134 f   srvclum:SRVCLUM.dll
 0001:00002144       PVRSRVPollForValue         00013144 f   srvclum:SRVCLUM.dll
 0001:00002154       SGXQueueTransfer           00013154 f   srvclum:SRVCLUM.dll
 0001:00002164       PVRSRVAllocDeviceMem       00013164 f   srvclum:SRVCLUM.dll
 0001:00002174       SGXCreateTransferContext   00013174 f   srvclum:SRVCLUM.dll
 0001:00002184       PVRSRVMapDeviceClassMemory 00013184 f   srvclum:SRVCLUM.dll
 0001:00002194       PVRSRVGetDCSystemBuffer    00013194 f   srvclum:SRVCLUM.dll
 0001:000021a4       PVRSRVEnumDCDims           000131a4 f   srvclum:SRVCLUM.dll
 0001:000021b4       PVRSRVEnumDCFormats        000131b4 f   srvclum:SRVCLUM.dll
 0001:000021c4       PVRSRVGetDCInfo            000131c4 f   srvclum:SRVCLUM.dll
 0001:000021d4       PVRSRVOpenDCDevice         000131d4 f   srvclum:SRVCLUM.dll
 0001:000021e4       PVRSRVCreateDeviceMemContext 000131e4 f   srvclum:SRVCLUM.dll
 0001:000021f4       PVRSRVEnumerateDeviceClass 000131f4 f   srvclum:SRVCLUM.dll
 0001:00002204       SGXGetClientInfo           00013204 f   srvclum:SRVCLUM.dll
 0001:00002214       PVRSRVAcquireDeviceData    00013214 f   srvclum:SRVCLUM.dll
 0001:00002224       PVRSRVEnumerateDevices     00013224 f   srvclum:SRVCLUM.dll
 0001:00002234       PVRSRVConnect              00013234 f   srvclum:SRVCLUM.dll
 0001:000022c4       WinMainCRTStartup          000132c4 f   corelib0:pegwmain.obj
 0001:000023c0       exit                       000133c0 f   corelib0:cexit.obj
 0001:000023d8       _exit                      000133d8 f   corelib0:cexit.obj
 0001:00002418       __GSHandlerCheckCommon     00013418 f   corelib0:gshandler.obj
 0001:00002454       __GSHandlerCheck           00013454 f   corelib0:gshandler.obj
 0001:00002478       __security_init_cookie     00013478 f   corelib0:seccinit.obj
 0001:000024d4       __security_check_cookie    000134d4 f   corelib0:armsecgs.obj
 0001:000024e8       __gsfailure                000134e8 f   corelib0:armsecgs.obj
 0001:0000252c       _initterm                  0001352c f   corelib0:crt0dat.obj
 0001:00002560       _cinit                     00013560 f   corelib0:crt0dat.obj
 0001:00002594       printf                     00013594 f   corelib1:COREDLL.dll
 0001:000025a4       free                       000135a4 f   corelib1:COREDLL.dll
 0001:000025b4       malloc                     000135b4 f   corelib1:COREDLL.dll
 0001:000025c4       memset                     000135c4 f   corelib1:COREDLL.dll
 0001:000025d4       _stricmp                   000135d4 f   corelib1:COREDLL.dll
 0001:000025e4       _isctype                   000135e4 f   corelib1:COREDLL.dll
 0001:000025f4       wcslen                     000135f4 f   corelib1:COREDLL.dll
 0001:00002604       _XcptFilter                00013604 f   corelib1:COREDLL.dll
 0001:00002614       __C_specific_handler       00013614 f   corelib1:COREDLL.dll
 0001:00002624       __security_gen_cookie2     00013624 f   corelib1:COREDLL.dll
 0001:00002634       __report_gsfailure         00013634 f   corelib1:COREDLL.dll
 0001:00002644       TerminateProcess           00013644 f   coredll:COREDLL.dll
 0001:0000266c       __IMPORT_DESCRIPTOR_COREDLL 0001366c     coredll:COREDLL.dll
 0001:00002680       __IMPORT_DESCRIPTOR_SRVCLUM 00013680     srvclum:SRVCLUM.dll
 0001:00002694       __NULL_IMPORT_DESCRIPTOR   00013694     coredll:COREDLL.dll
 0002:00000000       __imp_ReleasePowerRequirement 00014000     coredll:COREDLL.dll
 0002:00000004       __imp_NKDbgPrintfW         00014004     coredll:COREDLL.dll
 0002:00000008       __imp_FormatMessageW       00014008     coredll:COREDLL.dll
 0002:0000000c       __imp_GetLastError         0001400c     coredll:COREDLL.dll
 0002:00000010       __imp_SetPowerRequirement  00014010     coredll:COREDLL.dll
 0002:00000014       __imp_WideCharToMultiByte  00014014     coredll:COREDLL.dll
 0002:00000018       __imp___report_gsfailure   00014018     corelib1:COREDLL.dll
 0002:0000001c       __imp___security_gen_cookie2 0001401c     corelib1:COREDLL.dll
 0002:00000020       __imp___C_specific_handler 00014020     corelib1:COREDLL.dll
 0002:00000024       __imp__XcptFilter          00014024     corelib1:COREDLL.dll
 0002:00000028       __imp_wcslen               00014028     corelib1:COREDLL.dll
 0002:0000002c       __imp__isctype             0001402c     corelib1:COREDLL.dll
 0002:00000030       __imp__stricmp             00014030     corelib1:COREDLL.dll
 0002:00000034       __imp_memset               00014034     corelib1:COREDLL.dll
 0002:00000038       __imp_malloc               00014038     corelib1:COREDLL.dll
 0002:0000003c       __imp_free                 0001403c     corelib1:COREDLL.dll
 0002:00000040       __imp_printf               00014040     corelib1:COREDLL.dll
 0002:00000044       __imp_TerminateProcess     00014044     coredll:COREDLL.dll
 0002:00000048       \177COREDLL_NULL_THUNK_DATA 00014048     coredll:COREDLL.dll
 0002:0000004c       __imp_PVRSRVEnumDCFormats  0001404c     srvclum:SRVCLUM.dll
 0002:00000050       __imp_PVRSRVEnumDCDims     00014050     srvclum:SRVCLUM.dll
 0002:00000054       __imp_PVRSRVOpenDCDevice   00014054     srvclum:SRVCLUM.dll
 0002:00000058       __imp_PVRSRVCreateDeviceMemContext 00014058     srvclum:SRVCLUM.dll
 0002:0000005c       __imp_PVRSRVEnumerateDeviceClass 0001405c     srvclum:SRVCLUM.dll
 0002:00000060       __imp_SGXGetClientInfo     00014060     srvclum:SRVCLUM.dll
 0002:00000064       __imp_PVRSRVAcquireDeviceData 00014064     srvclum:SRVCLUM.dll
 0002:00000068       __imp_PVRSRVEnumerateDevices 00014068     srvclum:SRVCLUM.dll
 0002:0000006c       __imp_PVRSRVConnect        0001406c     srvclum:SRVCLUM.dll
 0002:00000070       __imp_PVRSRVGetDCSystemBuffer 00014070     srvclum:SRVCLUM.dll
 0002:00000074       __imp_PVRSRVMapDeviceClassMemory 00014074     srvclum:SRVCLUM.dll
 0002:00000078       __imp_SGXCreateTransferContext 00014078     srvclum:SRVCLUM.dll
 0002:0000007c       __imp_PVRSRVAllocDeviceMem 0001407c     srvclum:SRVCLUM.dll
 0002:00000080       __imp_SGXQueueTransfer     00014080     srvclum:SRVCLUM.dll
 0002:00000084       __imp_PVRSRVPollForValue   00014084     srvclum:SRVCLUM.dll
 0002:00000088       __imp_PVRSRVFreeDeviceMem  00014088     srvclum:SRVCLUM.dll
 0002:0000008c       __imp_SGXDestroyTransferContext 0001408c     srvclum:SRVCLUM.dll
 0002:00000090       __imp_PVRSRVUnmapDeviceClassMemory 00014090     srvclum:SRVCLUM.dll
 0002:00000094       __imp_PVRSRVDestroyDeviceMemContext 00014094     srvclum:SRVCLUM.dll
 0002:00000098       __imp_PVRSRVCloseDCDevice  00014098     srvclum:SRVCLUM.dll
 0002:0000009c       __imp_SGXReleaseClientInfo 0001409c     srvclum:SRVCLUM.dll
 0002:000000a0       __imp_PVRSRVDisconnect     000140a0     srvclum:SRVCLUM.dll
 0002:000000a4       __imp_PVRSRVGetDCInfo      000140a4     srvclum:SRVCLUM.dll
 0002:000000a8       \177SRVCLUM_NULL_THUNK_DATA 000140a8     srvclum:SRVCLUM.dll
 0002:000000ac       __security_cookie          000140ac     corelib0:seccinit.obj
 0002:000000b0       __security_cookie_complement 000140b0     corelib0:seccinit.obj
 0002:000000b4       pfnRegisteredWndProc       000140b4     wince_unittests.obj
 0002:000000b8       _exitflag                  000140b8     corelib0:cexit.obj
 0002:000000bc       __onexitend                000140bc     <common>
 0002:000000c0       __onexitbegin              000140c0     <common>

 entry point at        0001:000022c4

 Static symbols

 0001:00000d6c       GetString                  00011d6c f   sgx_blit_test.obj
 0001:0000224c       WinMainCRTStartupHelper    0001324c f   corelib0:pegwmain.obj
 0001:000022f8       doexit                     000132f8 f   corelib0:cexit.obj
